:020000022000DC
:10600000000001203D6202009562020097620200DA
:10601000996202009B6202009D6202000000000083
:106020000000000000000000000000009F6202006D
:10603000A162020000000000A3620200A56202004B
:106040009D870200AB620200D98B0200AF620200A2
:10605000B1620200B3620200558A0200B762020018
:10606000B9620200BB620200BD620200BF620200B0
:10607000C1620200C3620200C5620200C762020080
:10608000C96202000D700200CD620200CF62020000
:10609000A9700200D362020039B70200D762020081
:1060A000D9620200DB620200DD620200DF620200F0
:1060B000E1620200E3620200A7620200A76202003E
:1060C000E5620200E7620200E9620200EB620200A0
:0C60D000ED620200EF620200F1620200CB
:1060DC00364937480A1A02D0072291438D46354972
:1060EC0035480A1A06D00722914381F30988022207
:1060FC0082F3148831483249324A00F045F832486C
:10610C003249334A00F040F832483349334A00F000
:10611C003BF833483349344A00F036F833483449B5
:10612C00344A00F031F834483449354A00F02CF840
:10613C0034483549354A00F027F8354835490022AE
:10614C0000F02DF834483549002200F028F8344886
:10615C003449091A082903DB00220260043001606B
:10616C00314A90471F482049884205D002680430C4
:10617C0003B4904703BCF7E700208646EC460020AA
:10618C0000212A4A9047FEE7884207D0521A05D0D0
:10619C00037801300B700131013AF9D17047884214
:1061AC0002D002700130FAE77047000000000120B5
:1061BC0000E000200000012000000120B0D402000B
:1061CC00D82A0020502B0020F4620200F462020056
:1061DC0004C50200B0D40200D82A0020D82A00201E
:1061EC005CC602005CC602005CC602005CC6020013
:1061FC005CC602005CC602005CC602005CC6020003
:10620C00B0D4020028D50200502B0020502B0020C7
:10621C00502B0020E83A0020E83A0020E83A002011
:10622C00E83A0020E85A002061620200959D0200C5
:10623C000F484FF00701884385460E4880470E48AB
:10624C00016841F470010160BFF34F8FBFF36F8F92
:10625C00FFF73EBF09480A490A4A884207D0521A3A
:10626C0005D0037801300B700131013AF9D1704738
:10627C00000001209581020088ED00E01CC60200A0
:10628C00982A0020D82A0020FEE7FEE7FEE7FEE76A
:10629C00FEE7FEE7FEE7FEE7FEE7FEE7FEE7FEE7CA
:1062AC00FEE7FEE7FEE7FEE7FEE7FEE7FEE7FEE7BA
:1062BC00FEE7FEE7FEE7FEE7FEE7FEE7FEE7FEE7AA
:1062CC00FEE7FEE7FEE7FEE7FEE7FEE7FEE7FEE79A
:1062DC00FEE7FEE7FEE7FEE7FEE7FEE7FEE7FEE78A
:0862EC00FEE7FEE7FEE700BF3C
:1062F400704770477047000007B5044B0093044A89
:10630400402300F032F803B05DF804FB1963020087
:10631400512B00202DE9F84389461446E2B10F4B76
:106324000F4E0325002743F00108224609EB07011D
:10633400002003F0CBFE0744241A48B933785BB13C
:106344004FF47A40C047013D02D13570BDE8F8836F
:1063540001233370002CE8D1BDE8F88360C6020045
:10636400502B0020704703F0E5BEF0B595B01C46F5
:1063740008460D46164601F0E4FD1A9B09940024D4
:106384000D930822234605A9284608960A948DF8F9
:106394002C400C9401F013FE079B0293BDF81830B7
:1063A400ADF80C30BDF81A30ADF80E309DF814304D
:1063B4008DF8114003F00302012A1DD1BDF81440E9
:1063C400059EC3F3C203C4F383148DF81030A200F6
:1063D40008230EA9284601F0F2FDC6F3952608AB62
:1063E4000093224602AB0EA9304600F06BFB284610
:1063F40001F0ABFD15B0F0BD022AF8D1BDF816408E
:10640400C3F3C203C4F389148DF810300827082C91
:10641400264628BF08263B4632460EA9284601F0E8
:10642400CEFDA41B08AB02AA31460EA8374400F0E7
:10643400ADFB002CEBD1DAE710B5054CFFF793FF69
:106444000421204600F0AEFA0123637210BD00BFA0
:10645400D82A0020037813F0030F10B503F00404C6
:1064640002D004F0FF02F4B1B4B103F00303012B32
:1064740003D0022B09D0012010BD0A680088023223
:10648400C0F3831002440A60F5E70B6842880233C4
:1064940003EB92130B60EEE70B684288013303EBC6
:1064A40092130288F4E7104610BD00002DE9F04F66
:1064B40089B00646851C08A8494C019200230F4662
:1064C40000F8113D01F0ECF823683B606268A368B2
:1064D4001344226801339B1A04F21C4704F5836AAF
:1064E40004F21448AB421AD3019A0023002A6FD055
:1064F400012262F3010343F0040366F38913216864
:10650400A2689DF80F000A4003320D4444F822307B
:10651400256001F0E9F8012009B0BDE8F08F012100
:10652400384601F081F9504601F098F9404601F0EF
:1065340095F90DF120096068D4F808B049F8100DF8
:1065440000EA0B00033004EB80004946FFF782FFAA
:10655400049BB8B90BEA030204EB8202D1680591EB
:106564009A1C013303EA0B0B04EB8B0E0492DEF846
:106574000C30069301F00303012B21D0022B04D02D
:1065840083460CE00BEA0300DCE7BDF81630BDF8E7
:106594001AB0C3F38913033302EB93030493404605
:1065A40001F05FF908B1049B63605946384601F075
:1065B4003BF96268A3681344226801339B1A91E78C
:1065C400BDF81430BDF81AB0C3F383131344E5E7E0
:1065D400022262F3010343F0040366F39F538EE740
:1065E400642C002008B50E4B0E48FF229A6000224E
:1065F400C3F818241A605A60C3F8142483F82024BA
:1066040001F056FC38B9084A084B09499B1ADB08C3
:1066140002469A4200D108BD21F822200132F8E74F
:10662400642C0020DCC502005CC50200DCC502004D
:10663400982A002030B50B4C79B10B4A0B49121B38
:10664400D20800239A4201D1002030BD01EB83051A
:106654006D88854202D00133F4E7034654F83300D1
:1066640030BD00BF5CC50200DCC50200982A0020D2
:10667400094B013903EBC000032909D8DFE801F015
:106684000A02040604207047007970474079704775
:1066940000207047022070475CC50200034B586815
:1066A4001B68C31A58425841704700BF642C00202D
:1066B4002DE9F04387B0FFF7F1FF0746002840F0CB
:1066C400E6807B4DC5F81804BFF34F8F6868AC684B
:1066D4000DF1180848F8100D2040033005EB800038
:1066E4004146FFF7B7FE029B064600285AD104EA4A
:1066F4000302991C013305EB8202234005EB83035B
:10670400D268DB68049302F00303022B0392029124
:106714005AD1BDF80E306748C3F389194F46502F3C
:10672400A8BF502767F38F1307F10801ADF80E30A7
:1067340001F0D6FB8046002800F0B08001F001FC97
:10674400082203A93346404601F00EFC029924EACC
:1067540001020132920097422FD9002A00F0998059
:106764002140D6B20331BF1B534C05EB8101FFB26C
:1067740008233246404601F0F7FB34B106F1080322
:106784003A462146404601F0EFFB029B09F103091A
:1067940003EB99030293D5F81834002B47D1D5F8AD
:1067A400104450E02A689A4204D86A60384607B018
:1067B400BDE8F08304EA03008FE70C40E11C0823E2
:1067C4003A4605EB8101DDE7012B67D1BDF80C30BA
:1067D4003848C3F38311062928BF062161F38913BE
:1067E40002318900ADF80C3001F07AFB80460028B4
:1067F40054D001F0A6FB3346082203A9404601F019
:10680400B3FBBDF80C20C2F38312B31C96424FEACB
:106814008303C0D202994A1C21400331029205EB42
:1068240081010422404601F09FFB0136E9E740461E
:1068340001F08BFBFFF732FF80F00100C7B2B5E730
:10684400637A73BB6468002CFAD1404601F07DFB87
:1068540006A800F8114D00F023FFD5F818340BB941
:10686400029B6B609DF8070000F03EFFE2E723689F
:1068740020469B6898476468002CF8D10F4B104958
:106884001888000440F0020000F074F8D2E70027F2
:106894008CE7FEB214460849174669E7D5F8104458
:1068A400EAE7236841461B6820469847CAE700BFC9
:1068B400642C0020DCC50200702C0020AC2A0020CF
:1068C40074C602002DE9F74F284C80460F469246C5
:1068D40001A9012218469B46A568FFF7E7FD88B386
:1068E400DDF80490002609F102025E4534D100214E
:1068F4001F4800F066FF80F3100009F101022A40EE
:1069040004EB8202000405EA0903033340EA184059
:10691400D06014F8232068F3C50204F8232034F867
:10692400232066F3891224F8232054F8232001211C
:1069340067F39F2244F8232061F301026FF382027C
:1069440004F8232094F820341BB1FFF7B1FE00288B
:10695400FBD103B0BDE8F08F02EA050104EB81012D
:106964005AF82630CB6001360132BEE7642C002091
:106974008030002000231A46FFF7A4BF13B502ACF1
:10698400012344F8042D2246FFF79CFF02B010BDFA
:1069940007B58DE80C0002236A46FFF793FF03B0A6
:1069A4005DF804FB0F4A30B5D2F8104400232146A9
:1069B40041B90372D2F810444CB9C2F810044160D2
:1069C400184630BD0D7A9D4205D04968F0E76268EB
:1069D40042606060F4E701330A2BE8D14FF0FF33E3
:1069E400EEE700BF642C0020084A38B50123D2F832
:1069F400104482F820341D4604B938BD23686572FA
:106A040020465B6898476468F6E700BF642C002062
:106A1400C38873B504460D4633B1144A0092144931
:106A2400144A284600F07EFF217A05291CD0637A97
:106A34004BB1A088FFF71CFE0F4B104953F82020E0
:106A4400284600F06FFF227A0D4BA08853F822608D
:106A54000021FFF7EFFD0B4903463246284602B0FA
:106A6400BDE8704000F05EBF02B070BDEFC602002A
:106A7400D7C60200CFC602009CC60200F4C60200BC
:106A840004C70200F7C60200037A052B10B50C46B2
:106A94000FD0437A23B1084A0849204600F042FF48
:106AA4000749204600F03EFF2046BDE8104000F0B4
:106AB4002EBF002AF8D0F3E7EFC60200F4C60200A6
:106AC400A6CD02002DE9F04385B01F460C9D00239E
:106AD40006460C46904695F80C902B73294638468A
:106AE400FFF796FFB8F1060F09D8DFE808F00412A3
:106AF400181F283340003146284600F013FF0022B7
:106B040029463846FFF7C0FF85F80C9005B0BDE86C
:106B1400F08322683146284600F004FFEFE794E84A
:106B24000C003146284600F0FDFEE8E7A368009318
:106B3400314694E80C00284600F0F4FEDFE7E368F1
:106B44000193A3680093314694E80C00284600F0B2
:106B5400E9FED4E723690293E3680193A3680093F1
:106B6400314694E80C00284600F0DCFEC7E7636970
:106B7400039323690293E3680193A3680093314666
:106B840094E80C00284600F0CDFEB8E708292DE96A
:106B9400F84F80460E4617461C4636D8002593F813
:106BA4000C901D7319461046FFF732FFDFF87CA0E6
:106BB400DFF87CB0AE422AD918F8052059462046A1
:106BC40000F0B0FE0135082DF4D11649DFF864B0A9
:106BD400204600F0A7FE0025AE421DD918F805A0F6
:106BE400504605F019F8002814BF52462E22594683
:106BF400204600F097FE0135082DEDD101222146F3
:106C04003846FFF741FF84F80C90BDE8F88F5146F1
:106C1400204600F087FED5E70349204600F082FEB7
:106C2400E9E700BFCAC60200C8C60200C6C6020021
:106C3400C0C60200CCC602002DE9F84FDFF8A4B0AC
:106C44000025254B1B78ECB2A34201D8BDE8F88F90
:106C5400224BD3F8008018F8349001204A460021D2
:106C640004F0D0FEDBE9002300EA020601EA030790
:106C74003E4308EBC40A2CD023EA010122EA0000B7
:106C8400CBE90001484601F0D9FE18F834408146AA
:106C940022460120002104F0B5FE114BD3E9006720
:106CA400224606400F404846002104F0ABFE8F42C6
:106CB40008BF86420DD1DAF8043053B19AF80110B6
:106CC4004A1E51425141A1EB090041424141204633
:106CD40098470135B5E700BF88300020C030002058
:106CE400B0300020B83000202DE9F84307461F4893
:106CF40000F0B4FB002837D13A460120002104F00B
:106D040081FE1B4B04460D46D3E9000104EA00084A
:106D140005EA010958EA09021E461FD1384601F066
:106D24008DFE144B98B1D3E9000120432943C3E9F4
:106D34000001D6E900231D430F4B0C481968144386
:106D4400C6E900450022BDE8F84300F041BBD3E9A1
:106D5400000120EA040021EA0501E8E720EA04042E
:106D640021EA0505C3E90045BDE8F8839030002019
:106D7400B8300020B03000208C300020042AF7B551
:106D840005460C46164638D901F094FDC8B11C4B93
:106D94001C491D601C4B1D4F1C701D4B00221E60A6
:106DA4000023C1E900231B49C1E90023013CE4B2EB
:106DB4000026FF2C0BD1184A1848002100F0F6FADF
:106DC40003E001F03FFD0028E1D003B0F0BD23B2A1
:106DD40005EBC302032192788DF804108DF8052089
:106DE40001A93A4615F833008DF8066001F06CFDF0
:106DF400013CE4B20028DCD0E7E70720E5E700BF68
:106E0400C0300020B030002088300020ED6C02003B
:106E14008C300020B83000203D6C020064C70200B2
:106E240070B5084D084E00242B789C4201D30020F5
:106E340070BD3368012113F8340001F0B9FD013449
:106E4400F2E700BF88300020C03000201FB50021C9
:106E5400039001AA44F201000191029100F004F8A8
:106E640005B05DF804FB000010B572B6FFF7BCFD79
:106E7400FFF71EFC0028FBD1104C114920880004A8
:106E840040F00100FFF776FD0E4B1B68DB0700D5D1
:106E940000BE20880C49000440F00200FFF76AFDA0
:106EA400BFF34F8F09490A4BCA6802F4E0621343E7
:106EB400CB60BFF34F8F00BFFDE700BFAC2A0020BB
:106EC40068C70200F0ED00E074C7020000ED00E0C6
:106ED4000400FA0549B152B1531E1A4007D1826029
:106EE40001608380C260104670470E2070470920FD
:106EF400704710B58468C2688388121B934208D314
:106F0400C26813400268D154C3680133C3600020CF
:106F140010BD042010BD8268C3689A420AD08268FA
:106F2400838813400268D35C0B70836801338360E9
:106F34000020704705207047094A5378917801333F
:106F4400DBB2994208BF0023117899421FBF037036
:106F54005078182303FB002014BF0430002070472E
:106F6400C430002073B5054602A8002400F8014D82
:106F74000E4600F095FB0DF10600FFF7DDFF90B122
:106F840006700A4B9DF8062045605A709DF807006C
:106F940000F0AAFB24B9064B4FF48012C3F8002179
:106FA400204602B070BD0424F0E700BFC4300020C6
:106FB40000E100E0024B4FF43C6043F0010318474A
:106FC40090C7020038B50C4B0C4C4FF40032C3F898
:106FD400802001254FF48033C4F84833C4F80833C3
:106FE4006560FFF7E7FF064BA56000241C60FFF710
:106FF400E1FF044B1C7038BD00E100E000100140CB
:10700400E0310020D1310020F8B51F4B1F491B6827
:107014000025C1F84051C1F84451C1F84851C1F8A4
:107024004C51C1F80051C1F804514BB3D1F8044597
:1070340017490968641A24F07F442F461A68A2424B
:1070440009D8A41A15441A7CDE691AB11F745A6946
:1070540098699047AEB90F4B0F4A197813788B4251
:1070640005D10133DBB2022B08BF00231370127861
:107074000A4B43F822500A4B4FF48012C3F8002104
:10708400F8BD3346DAE700BFE431002000100140C8
:10709400E0310020DC310020DD310020D43100203B
:1070A40000E100E02DE9F74F9C4A9D4913780978E7
:1070B4009C4E994257D00133DBB2022B08BF002308
:1070C400137099491278994B0F6853F822003B18B2
:1070D40023F07F4300220B6033681546144696461E
:1070E40013B942B1336006E01968814229D902B16B
:1070F4003360091A19604FF0010833688C4FDFF8C8
:107104003CB200934FF00009002D61D02C46ED698C
:10711400854B60681A68831A23F07F41854B994236
:10712400A36800F2B7800B44236000236360A3606C
:10713400E361336801222274002B40F0B380346091
:10714400E2E7401A0C44D968C3F800E0D3F81CC045
:1071540031B13A1922F07F42DD615A6099601D46CF
:1071640063460122BCE70025A846C6E7531CB9784C
:10717400DBB299423B704FF0180303FB027208BF65
:107184003D7013799468022B1BD0032B11D0012B73
:107194001ED1217CE1B9D36863601369A36053698C
:1071A400E3609369A361644B1B78002BB0D06160EA
:1071B400AEE7002335681A46002D67D143B1356028
:1071C40006E0326813469246002B5AD100232374FA
:1071D4003A787B789342C9D1B9F1000F06D133686C
:1071E400009A9A4202D1B8F1000F44D03368002BC0
:1071F40073D0D3F800A0514D4B4BD5F804751C68DF
:10720400DFF840813E1B98F8003026F07F460336B5
:107214009BB94FF48033C5F84433C5F80433484B65
:107224004FF400324FF00109C3F880211A60C5F809
:107234000090FFF7BFFE88F80090B2452CBF54447D
:10724400A41924F07F44C5F84045D5F80435DB1B68
:1072540023F07F43E41B033324F07F44A3420AD981
:10726400D5F80435C5F84035FFF7A4FE344B4FF488
:107274000032C3F80021304B00221A7003B0BDE87D
:10728400F08F9C422CD09A46DB699DE72A74012337
:10729400ED6991E7121A22F07F429A4234BF9B1A99
:1072A400002341E7226819688A420BD88A1A1A60B7
:1072B400E36144E7521AD969184661B92260E16171
:1072C400DC6121E7184619689142F3D3891A1960E1
:1072D40019460346F2E70B46F5E7FFF773FECAE7E4
:1072E40054450DD1D369336053B90F48019201213C
:1072F400CBF808100360104B1970FFF75BFE019A7E
:10730400E1692368CAF81C1011B1086803440B60D2
:1073140033689A4218BF4FF0010957E7DC31002067
:10732400DD310020E4310020E0310020D4310020A0
:10733400C4300020FEFF7F00D03100200010014047
:1073440000E100E0D131002008B5FFF73BFE114B0E
:1073540000200B2218709A7058700F4B18600F4B56
:1073640018700F4B18700F4B4FF48012E021C3F8C4
:10737400802183F814131A6002F18042A2F56F226F
:10738400C2F8080583F81113074BD2F804251A60D4
:1073940008BD00BFC4300020E4310020DC310020EF
:1073A400DD31002000E100E0E0310020074B9B7854
:1073B4004BB132B128B10368187C20B959745A61B1
:1073C4007047072070470820704700BFC430002072
:1073D4002DE9F7431E4FBB7805460E469046ABB3E6
:1073E400A0B3042930D9436983B3437C02A80024A1
:1073F400012B00F8014D0CBF8946A14600F050F95D
:107404000DF10600FFF798FDE0B101230370114B65
:107414004560D3F8043583609DF80630C660C0F833
:107424001090C0F814807B709DF8070000F05CF9A0
:1074340024B9094B4FF48012C3F80021204603B04D
:10744400BDE8F0830424EFE70724F7E70824F5E711
:10745400C43000200010014000E100E0064A9278A8
:107464003AB130B1426922B1002202740221FFF71D
:1074740079BD0820704700BFC43000200648074A81
:1074840003780749D35C012213B1043001F0FCBF37
:107494000C3001F0CDBD00BFE42A0020683200208A
:1074A400103200200648074A03780749D35C0122BA
:1074B40013B1043001F096BF0C3001F061BD00BF80
:1074C400E42A0020683200201132002037B5057804
:1074D400012D04D035D3022D28D003B030BD43682C
:1074E4001F4C19782046FFF704FD78B11D4B01901D
:1074F4008DF800501B6868469847A168E368A28825
:107504005B1A9A420ED3FFF7B9FFE6E7A268E36875
:107514009A42F2D002AB134A03F8080D12681846D7
:107524009047EAE7104B01221A70D6E7C36801932B
:107534008DF80050FFF7A2FF0A4B1B686846984776
:10754400CBE70A490A48FFF7E6FC10B9FFF7AAFFA0
:10755400C3E702A8032300F8083D024B1B68EEE7CB
:10756400EC310020E8310020FC31002011320020F1
:1075740000320020F0B51F46234B89B006461A603E
:107584000C4600293DD08A8820480968FFF7A2FCF0
:10759400002834D1A289A1681D48FFF79BFC00286C
:1075A4002DD11C4D0FCD6C460FC495E80F0084E817
:1075B4000F0073690693337C174A18488DF81C70C2
:1075C400003318BF01238DF81430737C002B14BFD3
:1075D4000E2300238DF81530F3680293B3680393E8
:1075E4003368019369467368009301F05FF830B91A
:1075F4000B4B18703368013301D0FFF73FFF09B01C
:10760400F0BD0720FBE700BFE8310020EC3100208B
:107614000032002098C70200D1740200E42A00203E
:10762400FC31002070B5084C014608482678FFF765
:1076340072FC054636B100232370FFF71FFF08B123
:10764400FFF704FC284670BDFC310020EC3100201B
:1076540010B501460E48FFF74CFC0446A8B90D4886
:107664000D4A0378D35C63B1043001F001FF60B9C3
:107674000A490748FFF74FFC38B9BDE81040FFF747
:1076840011BF0C3001F0C8FCF1E7204610BD00BF6B
:1076940000320020E42A0020683200201132002049
:1076A40070B5EFF3108672B60C4A946801239CB946
:1076B40093600B4B0B4DD3F8801029401160C3F835
:1076C4008050D3F8841051604FF0FF32C3F8842007
:1076D400047006B962B670BD0370FAE71432002074
:1076E40000E100E0FC06FFBD084B9A6810B55AB1F2
:1076F40050B9EFF3108272B605491C680C605C68DF
:107704004C60986002B962B610BD00BF143200200C
:1077140000E100E037B550E8023F1FFAA3F5C48842
:10772400A54202BFBFF32F8F00220DE0C489254478
:107734008489A54228BF2D1BC3EA054540E80254AD
:10774400002CE8D14FF001028DF803200193019B36
:107754009DF803200B6002F0FF0322B14B88006800
:10776400184403B030BD1846FBE70A884B889A4298
:1077740009D150E8022FC2EA224240E80223002B3A
:10778400F7D1012070470020704701F01F024B0918
:107794000121914000EB830000F01FB801F01F03AA
:1077A40001229A404B0900EB8300D14300F02FB82B
:1077B4004B0901F01F0150F82300C84000F00100FC
:1077C400704700B550E8002F0B4640E8003E9EF09D
:1077D400000FF7D110465DF804FB00B550E8003FF8
:1077E40043EA010240E8002E9EF0000FF6D1104655
:1077F4005DF804FB00B550E8002F02EA010340E8FD
:10780400003E9EF0000FF6D110465DF804FB00B573
:1078140050E8003F03EA010240E8002E9EF0000F0A
:10782400F6D110465DF804FB00B550E8003F03EBC9
:10783400010240E8002E9EF0000FF6D110465DF8DC
:1078440004FB00B550E8003FA3EB010240E8002E22
:107854009EF0000FF6D110465DF804FB0121FFF7FE
:10786400BCBF0021FFF7C6BF10B590B14268836862
:1078740001689B1ADBB20A60013BDBB2FF2B026892
:1078840002D10020107110BD11684C1C14600B70E3
:10789400F2E70E2010BD37B5054602A8002400F813
:1078A400014DFFF7FDFE2A686B68116899420ED9F5
:1078B400481E106011F8014CEB68A98A01FB0434DE
:1078C400AB6811791B1ADBB2994238BF13719DF86A
:1078D4000700FFF709FF204603B030BD37B5054662
:1078E40002A8002300F8013D0C46FFF7D9FE2A68E0
:1078F4001368591C1160E968641AA98AB4FBF1F48D
:107904001C709DF80700FFF7EFFE03B030BD8268DE
:1079140010B504462AB143690168006998470023F9
:10792400A36010BD0EB403B5039929B102AA04AB38
:1079340042F8043D00F06CF802B05DF804EB03B0CB
:107944007047826830B40468551C8560A15482680D
:1079540043689A4202D330BCFFF7D9BF30BC7047AA
:107964002DE9F84F0A9C99460B9B17468246884698
:107974000A460126BA420FD24E4538BF4E4613F08E
:10798400010B01D164B900240125B9F1010F1AD901
:1079940009F1FF397D43F8E7B2FBF7F20136E9E775
:1079A4009B070ED5B9F1000F0CBF30252025A64248
:1079B400EAD2013C29465046FFF7C3FF002CF6D11A
:1079C400E1E72025F3E7B8FBF5F39F42E2D9DFF8BE
:1079D4003C90B8FBF5F3504619F8031005FB1388E7
:1079E400FFF7AFFFB5FBF7F5002DF2D1BBF1000FA8
:1079F4000AD03CB9BDE8F88F013C20215046FFF77E
:107A0400A0FF0CB1A642F7D3BDE8F88FB8C70200B7
:107A14002DE9F74F054617460C46002900F035813D
:107A240014F8011B49B92B7B002B00F02E8128464A
:107A340003B0BDE8F04FFFF76ABF252940F021816C
:107A440023460026194611F8012B2D2A24D0302A6A
:107A540026D02B2A27D000242A2A994603F1010193
:107A640024D13B681A1D1B683A601C44894699F866
:107A740000302E2B25D109F101014FF00008894671
:107A840011F8012BA2F1300009281CD80A2303FBAA
:107A94000823A3F13008F2E746F001060B46D1E7CC
:107AA40046F00206FAE746F00406F7E71A780B46B2
:107AB400A2F130010929DAD80A2101FB0424303C5F
:107AC400CAE74FF0000899F8001001F0FB02682A99
:107AD40002D119F8011FF8E769290FD04BD85829AA
:107AE40065D007D825296ED009F101042378002B2D
:107AF40096D198E7632962D06429F5D13A68D2F81F
:107B040000A0111D8AEAEA723960A2EBEA724FF012
:107B1400010B092A5BDCC34538BFC3462CB1BAF15B
:107B2400000F01DB710700D5013CB20702D5B8F1A3
:107B3400000F04D0F30702D4002C4ED10024BAF174
:107B4400000F52DACAF1000A2D212846FFF7F9FE88
:107B540006F00302022A05D1B8F1000F02D1002C6D
:107B640047D100248DE8500043460A225146284656
:107B7400FFF7F6FEB8E773294CD014D87029B3D1B7
:107B84003B681A1D3A60302128461C68FFF7D9FE6D
:107B940078212846FFF7D5FE00230193082300939C
:107BA40010222146E3E775292BD078299CD1396826
:107BB4000A1D3A6043468DE85000102228E03B68D5
:107BC4001A1D19783A602846FFF7BBFE8CE70A2392
:107BD4000BF1010B92FBF3F29BE7A345AFD22021FB
:107BE4002846013CFFF7ADFEA6E77007B0D52B2170
:107BF400ABE7A345B6D230212846013CFFF7A1FEEE
:107C0400ADE739680A1D3A608DE8500043460A2200
:107C14000968ACE73B681A1D3A60F107D3F800A085
:107C240012D55646A6EB0A0B16F8011B41B95C4562
:107C34007FF65AAF20212846013CFFF782FEF6E783
:107C44002846FFF77EFEEDE7BAF1000F11D050464B
:107C540004F098F80646B44200D964B90AF1FF3A30
:107C64001AF8011F00293FF43FAF2846FFF769FEC9
:107C7400F6E75646EFE720212846013CFFF761FE70
:107C8400E9E72846FFF75DFE30E703B0BDE8F08F73
:107C940070B508B10368B3B90D4D0E4B14225B1BCC
:107CA4000024B3FBF2F302FB03F6A64201D1002049
:107CB40070BD2B5928190BB91434F6E7DB699847C2
:107CC4000028F9D070BDDB69BDE87040184700BFDB
:107CD400D82A0020D82A002029DF704728DF7047DF
:107CE40070B503689D6886B004460E466DB11822CF
:107CF4000021684603F0F0FFA368059323790196F9
:107D04002BB1012B0DD06846A84706B070BD0123E6
:107D14008DF8003023690293E36803936369049345
:107D2400F1E702238DF80030E3681B030293F5E7C3
:107D3400034B187A0122B0FA80F05A744009704754
:107D44002032002070B5244D244E2B7A2C463BB9AA
:107D540023492448FFF7DEFC306008B9686070BD31
:107D64000223237233681A7972B1012A24D0184687
:107D74000321FFF7B5FF00232372636018491948F4
:107D8400BDE87040FFF7F1BC98695A69D9681D696C
:107D9400121AB2F5805F28BF4FF480529208012A6C
:107DA400014438BF01222844FFF796FF50B111283F
:107DB400DDD10123237270BDD8681A691044FFF71E
:107DC4008DFFF3E7237C2BB90146BDE87040022008
:107DD40000F00AB870BD00BF203200203832002005
:107DE40034320020F82A002038B5831E012B45D8F0
:107DF400234C237A002B41D0022B09D1032830D005
:107E0400204B1B680022E2601A793AB1012A22D081
:107E1400637C7BBBBDE83840FFF794BF9A6959691E
:107E24008D1AB5F5805F94BF521902F580529A619C
:107E34009142EDD102284FF0000308BF1946237286
:107E4400104B18BF0D211868FFF74AFF0E490F4861
:107E5400FFF78BFCDCE71A6901321A615B699A420D
:107E6400E7E7E3680133082B01D8E360D0E7002398
:107E7400E360DFE7BDE8384003F032BC38BD00BF43
:107E8400203200203832002034320020F82A00202A
:107E940000F0FD03012B08D1044B00225A74421E4A
:107EA400504250411874FFF74DBF704720320020F4
:107EB400FFF7DABCF8B546790446721E00239342F4
:107EC400246804D301460025B54202D3F8BD01332A
:107ED400F5E70F682046FFF701FD01353946F3E762
:107EE4002DE9F843878ACD1C8046FFF7D4FC043F74
:107EF4003D440446B5FBF7F5002650B10123EDB22D
:107F040006714371C780013DC0F800808146AE42CE
:107F140002D32046BDE8F8834046FFF7BCFC074681
:107F240048B16379013363710136C9F80000C0F8C0
:107F340000808146EBE72046FFF7BCFF3846BDE8EA
:107F4400F88301210430FFF76FBC10B5012104460A
:107F54000430FFF776FC10F0FF0F04D12046BDE893
:107F64001040FFF7A7BF10BD2DE9F843C6880433BE
:107F74000F46B3FBF6F4154606FB143380463CB9B2
:107F8400A6EB0309A94528BFA9462DB9BDE8F88386
:107F9400D8F80080013CF2E7043308EB0300A5EBBA
:107FA40009054A46391903F06DFEAE424C44D8F82F
:107FB4000080B1464FF0000328BFA946E5E72DE94C
:107FC400F843C6880F46191D1546B1FBF6F48046E2
:107FD40006FB14113CB9A6EB0109A94528BFA94623
:107FE4002DB9BDE8F883D8F80080013CF2E70431EC
:107FF4004144A5EB09054A46381903F043FEAE4255
:108004004C44D8F80080B1464FF0000128BFA9467F
:10801400E6E741DF70470000064B10B500241C70F2
:10802400054B1C60BFF35F8F0449054800F030F82E
:10803400204610BD4432002048320020E4C702002C
:108044003C32002007B502A8002300F8013DFFF7E9
:1080540027FBF1EE103A23F09F03E1EE103ABFF351
:108064005F8F0A4B4022C3F884219DF80700FFF775
:108074003BFB03F045FB20B1FFF7CBFF03B05DF8FA
:1080840004FB20BF40BF20BFF8E700BF00E100E0D1
:108094000B684A684360934208BF0023016008BF2D
:1080A40043607047436843B10268916852680B4467
:1080B4009342436004BF0023436070470D4930B5C9
:1080C400A1F594720225914201D8002030BD8B1A8B
:1080D400DB1093FBF5F302EBC30452F83330834215
:1080E40005D802D204F10802EDE7606830BD2146EC
:1080F400E9E700BF34C9020008B5FFF7DFFF024B10
:10810400002808BF184608BDF9C7020010B5044688
:10811400C0B2FFF79DFA204610BD0000094B1B7842
:10812400062B0CD1084B1B681A0708D1074B18689B
:1081340000F0F000A0F1300358425841704700208D
:10814400704700BFE00F00F0E40F00F0E80F00F00C
:108154000C4B1B78062B10D10B4B1B681A070CD148
:108164000A4B186800F0F003302B08D000F0E00050
:10817400A0F1400358425841704700207047012045
:10818400704700BFE00F00F0E40F00F0E80F00F0CC
:1081940008B5FFF7DDFF28B17F4B804A1B68C3F3A6
:1081A40004231360FFF7BAFF10B17D4B7D4A1A60B8
:1081B400FFF7CEFF28B17C4B7C4A1B68C3F34233E4
:1081C4001360FFF7ABFF20B1794AD36823F08073C3
:1081D400D360FFF7BDFF40B14FF080430022C3F8E6
:1081E4000C21C3F81021C3F83825FFF797FF10B10D
:1081F400704B03221A60FFF791FF40B16E4B0522CA
:108204001A6001229A6700229A603F225A606B4BDF
:108214001B78062B09D16A4B1B68190705D1694BDA
:108224001B6803F0F003502B67D0FFF791FF28B1D0
:10823400654B664A1B6803F04F031360FFF788FF22
:1082440048B14FF08043D3F80024D20744BF6FF005
:108254000102C3F800245E4B1B68062B04D15D4B5E
:108264001B68062B00F091805B4AD2F8883043F4F7
:108274007003C2F88830BFF34F8FBFF36F8F4FF096
:108284001023D3F80022002A03DBD3F80432002B96
:108294002FDA524B0122C3F80425D3F80024002A14
:1082A400FBD04FF010221521C2F80012D3F800249D
:1082B400002AFBD04FF010231522C3F80422474BA9
:1082C4001A46D3F800140029FBD00021C3F8041582
:1082D400D2F80034002BFBD0BFF34F8F3E49404B04
:1082E400CA6802F4E0621343CB60BFF34F8F00BF50
:1082F400FDE73C4B3C4A1A6008BD4FF080523B4BB3
:10830400D2F80414C3F82015D2F80814C3F82415BD
:10831400D2F80C14C3F82815D2F81014C3F82C158D
:10832400D2F81414C3F83015D2F81814C3F834155D
:10833400D2F81C14C3F84015D2F82014C3F844151D
:10834400D2F82414C3F84815D2F82814C3F84C15ED
:10835400D2F82C14C3F85015D2F83014C3F85415BD
:10836400D2F83414C3F86015D2F83814C3F864157D
:10837400D2F83C14C3F86815D2F84014C3F86C154D
:10838400D2F84424C3F870254FE7194A136843F41C
:108394008063136068E700BF240300104035014088
:1083A40074C007400DF0ADBA440200103C05004013
:1083B400F0ED00E0A005004010560040E00F00F092
:1083C400E40F00F0E80F00F058020010E40E004043
:1083D400300100103401001000ED00E000E0014025
:1083E4000400FA050C2B00200090D00300C00040CC
:1083F4003C170040054A4FF0A043105CD3F8043505
:1084040023FA00F0C04300F001007047F2CC0200F0
:10841400044B1A5C012393404FF0A042C2F80C3580
:10842400704700BFF2CC0200044B1A5C0123934056
:108434004FF0A042C2F80835704700BFF2CC0200EA
:1084440008B50020FFF7F0FF0120FFF7EDFF022041
:10845400FFF7EAFF0320BDE80840FFF7E5BF08B5D2
:108464000020FFF7D5FF0120FFF7D2FF0220FFF71E
:10847400CFFF0320BDE80840FFF7CABF074A4FF00B
:10848400A041105CD1F804350122824022EA0300A5
:108494001340C1F80805C1F80C357047F2CC02004E
:1084A400054A4FF0A043105CD3F8103523FA00F0CE
:1084B400C04300F001007047EECC02000D2809D043
:1084C4000E2809D00F2809D010280CBF03204FF024
:1084D400FF3070470020704701207047022070472A
:1084E400014B185C704700BFEECC0200C20708B510
:1084F40001460CD54FF0A0430322C3F84427C3F828
:108504004827C3F84C27C3F85027FFF799FF8B0778
:108514000AD54FF0A0430C22C3F83427C3F83827F8
:10852400C3F83C27C3F8402708BD000038B5084C01
:1085340004F108030546002818BF1C4623682BB124
:108544001A6822605B6828469847F7E738BD00BF81
:108554005432002020B9054B01225A70FFF7E6BFC0
:10856400012802D1014A9070F8E770474C3200208C
:1085740020B9034B01225A70FFF7D8BF704700BFE0
:108584004C32002038B50B4C237883B90A48636019
:10859400A3602361E36000F0D1F8054603F0B0F86E
:1085A40008B900F0D9F801232370284638BD852581
:1085B400FBE700BF4C3200205985020037B502A802
:1085C4000023094C00F8013DFFF76AF8E368013B1A
:1085D400E360E56815B900F0D3F8A5709DF80700CD
:1085E400FFF782F803B030BD4C320020012813B5E8
:1085F40009D003D303281BD002B010BD0F4B0122B6
:10860400C3F88020F8E702A800230D4C00F8013DD0
:10861400FFF746F823780BB9FFF7B4FFE3689DF83A
:1086240007000133E3600123A370FFF75DF8E3E77C
:1086340000F092F8FFF7C2FFDEE700BF00E100E0C0
:108644004C3200201FB503788DF800304368019345
:10865400037A8DF80830C3680393054A054B6846CE
:1086640053F8213052F82110984705B05DF804FB07
:1086740060320020643200201FB503788DF800308A
:108684004368019383688DF80830C3680393054AEF
:10869400054B684653F8213052F82110984705B02D
:1086A4005DF804FB6032002064320020F0B5194B01
:1086B400067891F81DC043F82620174B96460A69A0
:1086C40043F82620154B03F806C00C4607460FCC8A
:1086D40089B06D460FC594E80F0085E80F00049635
:1086E400BCF1000F0AD0BEF1000F0D4A694608BF65
:1086F4000022381D00F0ACFD09B0F0BDBEF1000F42
:10870400084A694608BF002207F10C0000F076FB16
:10871400F2E700BF6432002060320020683200209B
:10872400498602007D86020000F180400023036038
:1087340082B003680193019B02B07047054A137924
:108744002BB90121106011715371184670478520AF
:10875400704700BF6C320020084B1A68D20706D459
:10876400E02283F800230122C3F880211A604FF02D
:1087740080430122C3F81825704700BF00E100E0E0
:10878400044B01221A604FF08042D2F81834DB0304
:10879400FBD470470C000040124B1B6810B573B13A
:1087A4004FF48070FFF7C0FF4FF080430122C3F8FD
:1087B40008230D4B587910B95A711B6898470B4B15
:1087C4001B6873B14FF48270FFF7AEFF4FF0804324
:1087D4000222C3F80823044B01201B68BDE81040A3
:1087E400184710BD000100406C3200200401004015
:1087F40000F1804000F5C040002382B003600368AC
:108804000193019B02B07047800000F1A040D0F8B2
:10881400003723F44033C0F80037D0F8003743EA78
:108824000141C0F800177047054B4FF0FF3207288D
:1088340043F8202084BF1B1883F84820704700BFEA
:108844007432002010B5174C94F8583043BBFF2104
:10885400E2180133202B82F83010F9D10021C8B27C
:10886400FFF7E2FF01310C29F9D1002104220E485F
:1088740003F032FA0D4BE02283F806234022C3F8BA
:1088840080214FF4BE701A60FFF7B2FF084B4FF01F
:108894000042C3F80423012384F85830002010BD9B
:1088A400082010BD74320020C832002000E100E02E
:1088B40000600040034B93F85800003018BF0120BB
:1088C400704700BF74320020F0B5374D2B1893F970
:1088D4003030002B65DA8E78C6F34006002E0BBFCD
:1088E400082300230C240824A34201D10420F0BD52
:1088F40055F82370013740D12F185CB287F8304007
:1089040045F8232016B92B4483F848008B785A077E
:1089140013D4DE0733D5830003F1A043D3F8002733
:1089240022F00202C3F80027204EC20800F0070715
:108934000123BB40B75C3B43B3548B780A7813F0F4
:10894400020325D0A30003F1804303F5C0430002D2
:10895400D3F8101521F4473121F44071C3F81015F0
:108964001204D3F8101500F4F85002F44032104306
:108974000843C3F810050020F0BD0133B4E74A787A
:1089840000F5E0734FF0A046920046F82320CBE7B1
:10899400083C2C4494F8500040EA821284F8502099
:1089A400E9E70820F0BD00BF74320020C83200207F
:1089B40038B5204C251895F93020072A18DD2244B3
:1089C40092F848309B09032B0DD14FF0A043D3F804
:1089D4001035C34013F0010F0CBF02210321BDE881
:1089E4003840FFF711BF012B14BF03210221F6E722
:1089F400D3B2072B1CD8930003F1804303F5C04383
:108A0400D3F8100540F00100C3F8100502F140004E
:108A1400800080B2FFF7ECFE51B195F9303054F884
:108A240023302BB1012303FA02F2034BC3F80423CE
:108A340038BD00BF74320020006000404FF0A043F6
:108A4400D3F8103523FA00F000F00100704700005D
:108A54002DE9FF4700245A4A5A4E5B4D01940121E7
:108A6400A2F5C04052F8043B012B80B206D1D6F8DF
:108A740004330B4202D0FFF7BBFE0C43AA424FEA79
:108A84004101EDD1514B1B68012B0AD14FF4BE704B
:108A9400FFF7AEFE4FF0A04344F00044D3F8103586
:108AA400019314F0FF0F38D1002C80F2858000234D
:108AB4000293DFF81C914FF0FF3303930126002447
:108AC400A0464FF0A04709EB080393F95020531C2C
:108AD40061D0D2B222F0C005E90804A8084402F02B
:108AE400070310F804EC06FA03F31EEA030F52D04E
:108AF40009EB050E92099EF930E059F82EA0BAF15F
:108B0400000F26D1032A46D10DF1080C1CF801E010
:108B14004EEA030E0CF801E01DE02D4F012600255E
:108B2400344210D0AB0003F1804303F5C043D3F8C3
:108B34001005D3F8101557F8253023B1C1F30141BE
:108B4400C0F3042098470135082D4FEA4606E7D1C3
:108B5400AAE7032AD8D005F5E07110F80C0C57F8F1
:108B640021101842C1F3014105D0022913D1032A6F
:108B74000BD1114604E003290DD1032A05D10221AA
:108B84002846FFF741FE0134E4B2BAF1000F02D0E7
:108B940011462846D04708F10108B8F1040F92D1D4
:108BA40054B14FF0A043019AD3F81035934203D047
:108BB4000193029B039382E704B0BDE8F08700BFF2
:108BC4000061004000600040206100407C61004082
:108BD40074320020014B1B68184700BFD0320020BC
:108BE4000D4B984237B50D4610D102A8002300F86A
:108BF400013DFEF755FD094B1C7914B901221D6096
:108C04001A719DF80700FEF76FFD14B9002003B038
:108C140030BD1120FBE700BF00200040D03200200F
:108C24000023435082B043580193019B02B0704724
:108C34000A4610B54FF48E71FFF7F2FF136A91687C
:108C4400C95C136A01331362C0F81C1510BD0246D7
:108C540008B54FF492710068FFF7E2FF4FF4847196
:108C64001068FFF7DDFF136801221A6008BD8B69E5
:108C74000A4610B54FF4847123B9FFF7D1FFD0F839
:108C8400183510BDFFF7CCFF536AD168D0F818052A
:108C9400C854536A0133536210BD00001FB5012349
:108CA4008DF80030044B02900191684693E8060069
:108CB400904705B05DF804FBD832002030B54D4A2A
:108CC400D2F8043313F4007F85B015464FD0D2F8A0
:108CD4002431002B4BD04FF492711046FFF7A0FFC4
:108CE4004FF40173C2F80833434B93F8291009B9C0
:108CF400012151603F4902228DF80020D1F88024DF
:108D0400C1F8802403929A690292DA6801920022DF
:108D14009A61DA61684693E8060090473548D0F8CE
:108D24001C315BB134490A6A4B699A420A464CD2F7
:108D340091F82830002B48D1FFF77AFF2D4AD2F85A
:108D4400443193B14FF4A2711046FFF769FF2A4BE7
:108D540093F8291009B1012111609A692AB10022FE
:108D64009A61586AD968FFF799FF05B030BDD5F804
:108D740004335B07D2D5D5F80831002BCED01E4C76
:108D84001C482146FFF773FF636AA2699A4223468F
:108D9400C4D1E26952B12369E168E3600023606AE7
:108DA400A261E3616362FFF779FFB7E794F82920D2
:108DB4000AB901226A600F4A4FF40171C2F808131C
:108DC40000229A61586AD968EDE74FF48E71094818
:108DD400FFF726FF51690029B0D000230291916862
:108DE4008DF8003001915361684692E80A00984773
:108DF400A4E700BF00200040D83200202DE9F8434A
:108E04005B4B047991462C2202FB0432064692F80D
:108E14002A200D469846002A40F0A580554900684E
:108E2400FFF7DEFE0746002840F09F80296833687C
:108E3400481C0BD04FF0A04001228A40C0F80825FE
:108E440001F5E0724FF0030E40F822E06868421C1E
:108E54001FBF00F5E0724FF0A04E4FF0000C4EF82B
:108E640022C0AA6995F814E0C3F824256A7DBEF1EE
:108E7400010F4EEA0202C3F86C25C3F81405C3F8C7
:108E84000C151DD1AA68511C1FBF02F5E0714FF0EB
:108E9400A0404FF0000E40F821E0E968481C0BD0D8
:108EA4004FF0A04E01208840CEF8080501F5E0708F
:108EB4004FF0030C4EF820C0C3F80815C3F8102572
:108EC4002C23634308EB0302C2F804902A6948F890
:108ED4000320B9F1000F33D04FF48E7130682D7F29
:108EE400FFF79EFE30684FF4A271FFF799FE3268D7
:108EF400214BC2F80433120B53B2002BA8BF03F169
:108F040060404FEA53134FEA4511BABF1B4802F0C1
:108F14000F0500F561404FEA8303B4BFC9B2C9B27B
:108F240003F16043B4BF415580F8001303F5614376
:108F340002F01F02012101FA02F2C3F880211A6033
:108F440033680422C3F800252C2303FB0483002286
:108F54009A61DA6183F829205A61012283F82A2070
:108F64003846BDE8F8830827FAE71127F8E700BF79
:108F7400D8320020C18C02008000020014ED00E011
:108F84002DE9F843234F06794FF02C0909FB0674A9
:108F940080466569002D37D16261A16025624FF476
:108FA4008E71006884F82850FFF73AFED8F8000064
:108FB400012383602146FFF73BFE6368A14633BB70
:108FC400D8F80050226A63699A4212D3D8F8003064
:108FD400D3F81C21002AFBD00122DA6000202C23C4
:108FE40003FB067600237361BDE8F88394F8283008
:108FF40043B9D5F81C31002BF8D049462846FFF771
:1090040017FEDFE70F20EAE71120BDE8F8832846C2
:10901400BDE8F883D83200200379044A2C2101FBEF
:1090240003235869003018BF01207047D83200204C
:109034002DE9F8433D4D07792C2303FB07530646DE
:109044005C6824B103684FF40170C3F808032C234F
:1090540003FB0753986940B3D869002862D024B150
:1090640033684FF40172C3F804231120BDE8F88378
:10907400002A44D1002C42D14146FFF7F8FDD9F82B
:109084002430D9F818209A422DD8224637E05A6065
:1090940045E033684FF40172C3F804233FE0032032
:1090A400BDE8F8830F20BDE8F8839A61D96058625F
:1090B400D8612C2404FB075393F829301BB910B949
:1090C4003046FFF7C4FD04FB07535B68002BE0D177
:1090D4004FF4A2713068FFF7A3FD4FF02C0907FB92
:1090E400045809FB07593068D0F82421D0F8083116
:1090F400D0F84441002BBBD10CB9002AF3D02C2367
:1091040003FB07550023AB61002AC8D1002CC9D149
:1091140095F82910336801220029B8D01A6000207C
:10912400BDE8F8831961DA610120C2E7D832002072
:109134000023435082B043580193019B02B070470F
:109144001FB501238DF80030054B8DF808000191FF
:10915400684693E80600904705B05DF804FB00BF3D
:10916400043300207FB5384AD2F82461002E49D058
:1091740010464FF49271FFF7DBFF02238DF80030A5
:10918400D2F88034C2F880340393D2F83C358DF899
:1091940008302E4BDA68019200229A61DA6168463F
:1091A40093E806009047284AD2F8443173B14FF44B
:1091B400A2711046FFF7BCFF244B996931B100211D
:1091C4009961D2F83C05D968FFF7BAFF1E4AD2F874
:1091D4002031ABB14FF490711046FFF7A9FF1B4B40
:1091E400596969B1D2F84C158DF8081000229968B4
:1091F4008DF8002001915A61684693E80600904773
:1092040004B070BDD2F81031002BCCD04FF488716B
:109214001046FFF78DFF0D4BD2F83C059969884243
:10922400C1D1DC696CB1D2F80052D96825F02005AF
:10923400C2F800521A699C61DA60DE61FFF780FFB0
:10924400B1E79C61D968F9E70020004004330020AD
:109254002DE9F8435F4B06799146242202FB06323E
:10926400044692F820200D469846002A40F0AD802E
:1092740059490068FFF7B4FC0746002840F0A7806E
:1092840029682368481C0BD04FF0A04001228A4073
:10929400C0F8082501F5E0724FF0030E40F822E013
:1092A4006868421C1FBF00F5E0724FF0A04E4FF0FB
:1092B400000C4EF822C0AA6995F814E0C3F82425DE
:1092C4006A7DBEF1010F4EEA0202C3F86C25C3F8B1
:1092D4000C15C3F814051DD1AA68511C1FBF02F553
:1092E400E0714FF0A0404FF0000E40F821E0E96833
:1092F400481C0BD04FF0A04E01208840CEF8080542
:1093040001F5E0704FF0030C4EF820C0C3F80815C7
:10931400C3F810252423734308EB0302C2F8049016
:109324002A6948F80320B9F1000F3DD04FF4887141
:1093340020682D7FFFF7FCFE4FF490712068FFF743
:10934400F7FE4FF492712068FFF7F2FE20684FF4A5
:10935400A271FFF7EDFE2268204BC2F80433120B12
:1093640053B2002BA8BF03F160404FEA53134FEAF6
:109374004511BABF1A4802F00F0500F561404FEAE3
:109384008303B4BFC9B2C9B203F16043B4BF41554A
:1093940080F8001303F5614302F01F02012101FA72
:1093A40002F2C3F880211A6023680822C3F800255A
:1093B400242303FB068300229A61DA615A610122A5
:1093C40083F820203846BDE8F8830827FAE71127F8
:1093D400F8E700BF04330020699102001003020083
:1093E40014ED00E001F06043B3F1005F2DE9F041BA
:1093F400074632D11D4B0679242505FB06359846D0
:109404006C696CBB6A61A96000684FF49071FFF7E6
:109414008FFE4FF4AC713868FFF78AFE3B686A69C7
:10942400A968C3F84415C3F8482501229A606A68FC
:10943400CAB9D3F82011D3F8582149B9002AF8D071
:109444000F20242303FB068600237361BDE8F0810B
:10945400002A14BF0F200020F3E71020BDE8F0819C
:109464001120BDE8F0812046BDE8F08104330020DE
:109474000379044A242101FB03235869003018BFEF
:109484000120704704330020F8B501F06043B3F1C4
:10949400005F04460F4628D10379314E242101FB95
:1094A4000361486820B121684FF40475C1F808537A
:1094B400242101FB03639D69CDB1D96900294AD0F8
:1094C40020B123684FF40472C3F804231120F8BDBB
:1094D400D3F8002242F02002C3F800221DE04FF42A
:1094E4000472C3F804230020F8BD1020F8BD9A616B
:1094F400DF60DD614FF488712068FFF719FE4FF4D7
:10950400A2712068FFF714FE2368C3F83475C3F80A
:109514003825002DDCD101221A602279242101FB97
:10952400026149680029DAD1D3F81041D3F8441113
:10953400D3F8240114B909B90028F5D0242303FB76
:1095440002660023984214BF032018469942B3616F
:1095540018BF0F20F8BD1F61DA610125CAE700BFFB
:10956400043300200220FEF789BF000008B5094B30
:109574001B7853B10020FEF757FF0120FEF754FF7C
:109584000320BDE80840FEF74FBFBDE80840FEF7E2
:1095940057BF00BF29330020F8B5764C2378054621
:1095A4001BB100232370FFF7E1FF172D00F2838026
:1095B400DFE805F00C13133F5060717B83888388C8
:1095C400909494949494BEC2C9D0DADAFFF7CEFF93
:1095D400694B00241C702046F8BD0020FEF70AFFEA
:1095E400F8B10020FEF720FF022D0CBF4FF4E1611B
:1095F4004FF47A61604B1D704FF400404FF4FA74DD
:109604000025E0FB01454FF47A72002320462946E9
:1096140002F00CFA002201465848BDE8F840FDF774
:10962400D7BEFEF7F5FE022D0CBFC8214FF4C8715A
:10963400E0E70020FEF7DEFE40B10020FEF7F4FE76
:109644004FF4487103224C4B1A70D5E7FEF7E0FE45
:10965400C821F7E70020FEF7CDFE30B10020FEF769
:10966400E3FE4FF47A610422EDE7FEF7D1FE4FF4F6
:10967400C871F8E70020FEF7BDFE48B10020FEF7F0
:10968400D3FE3D4B05221A7041F69A110022C3E71E
:10969400FEF7BEFEF5E70020FEF7F0FE364B06228D
:1096A4001A70002240F6CD41B6E70020FEF7B0FE66
:1096B4000722314B1A7000248DE701202070FEF739
:1096C400DDFEEEE701202070FEF7D8FE00224FF405
:1096D4008041A1E7FEF7C3FE0C22EAE72848294EA1
:1096E400FDF7BCFED5F1110504461CD0D8B9012DF7
:1096F40013D0C8235D434FF4FA7000214FF40047A0
:109704004FF47A720023C7FB050102F08FF9224659
:1097140001461B48FDF75CFE04460220FEF778FE76
:109724000123337057E70220FEF77EFE0023F8E79B
:10973400FFF71CFF1222BCE7FFF718FF0020FEF71B
:1097440067FE1322B5E7FFF711FF0120FEF760FE65
:109754001422AEE7FFF70AFF0020FEF759FE0120AE
:10976400FEF756FE1522A4E7FEF779FE024B1D70A4
:10977400A1E700BF9C330020A43300206C330020F9
:109784002C330020293300202DE9F04781460D4673
:10979400FEF794FE0328044631D8012D04D022D3C9
:1097A400022D2ED0BDE8F087194D47003A18A918AC
:1097B400AE5C4A7852B1DFF86880164842464FF4EE
:1097C4000041FDF705FE08B988F800903B192B44C9
:1097D4009A78114B1A5596B1104B1B687BB13046E1
:1097E400BDE8F04718470B48FDF738FE084B04EB7B
:1097F400440213449E78084B1B5DB342EBD0BDE892
:10980400F087034B00EB40041C446678E3E700BF99
:109814008C3300204C330020A5330020A0330020DB
:109824002833002002210078FFF7AEBF044B1B68E9
:10983400DB0703D5034B1878FFF7AEBE704700BFB4
:1098440098330020A4330020032801D8FEF728BE53
:1098540000207047044B1B6813F0010301D0FFF78D
:109864009BBE1846704700BF9833002038B51C4B88
:1098740018601C4B10F00204054619601AD01A4BEC
:109884001A480E221A700F22DA7010229A711122CD
:109894005A72042140F26662FDF770FA044648B930
:1098A400FDF7BEFA044628B90146114A1148FDF7EE
:1098B4007DFD0446EB0711D50120FEF717FE6CB9B8
:1098C40021460D4A0D48FDF771FD044630B90C4A96
:1098D4000C480121BDE83840FDF768BD204638BD7D
:1098E40098330020A03300208C33002014CD0200D4
:1098F4002998020038CD0200319802003CCD0200C4
:109904006995020034CD0200032812D8012A0BD134
:10991400012908D100F10E02D2B200EB40000C4B39
:109924001A540020704700220129F6D009D30229D5
:1099340001D007207047064B00EB400018444270EA
:10994400EFE7034B00EB400018448270E9E700BFE7
:109954008C330020032808B512D8FEF7C1FD80001F
:1099640000F1A040D0F8003723F44033C0F80037AA
:10997400D0F8003743F44033C0F80037002008BD66
:10998400062008BD08B5012202210020FFF7BCFF14
:1099940008B1072810D1072202210120FFF7B4FFE4
:1099A40008B1072808D100210A220846FFF7ACFFB6
:1099B40010B1072808BF002008BD00000388102B41
:1099C40010B502D0112B1ED010BD194C2168B1B9AD
:1099D40001220846FFF798FF08B1072821D1072282
:1099E40002210120FFF790FF08B1072819D10422B2
:1099F40002210020FFF788FF08B1072811D123684E
:109A04000133236010BD0A4A1368013B136073B924
:109A1400FFF7B8FF58B1074B1B6843B1BDE81040CE
:109A24001847044B1B68002BE9D09847E7E710BDA3
:109A3400B0330020AC33002008B50020FFF78AFFC4
:109A440008B1062806D10120FFF784FF10B10628CB
:109A540008BF002008BD00000D4B10B518600C466F
:109A640029B10120FFF7F0FE40B102232370094B16
:109A74001B6853B9BDE81040FFF784BFFFF7E4FE4D
:109A840008B10B23F2E72070F1E7002010BD00BFFE
:109A9400AC330020B033002076DF70477ADF7047A4
:109AA4007CDF70477FDF70478FDF7047B1DF70471F
:109AB40033DF7047FDF7CAB908B50020FFF7CAFEC7
:109AC40008B1FDF7C3F9FFF7B7FF08B1FDF7BEF919
:109AD400FFF7EEFF18B1BDE80840FDF7B7B908BDC0
:109AE4000388212B13B5044637D01DD8112B26D05B
:109AF400132B3CD0102B2ED1254B2649188800045B
:109B040040F00300FCF736FF0720FFF7A3FE08B17F
:109B1400FDF79CF9204BA1882048198001F0DCFA5C
:109B2400C8B1FDF793F916E0522B28D0562B01D07B
:109B34003B2B10D11321A088FFF7AEFFF0E7144BA5
:109B440017491888000440F00300FCF713FF124B78
:109B54004FF6FF721A8002B010BD002301A980885D
:109B64008DF804308DF80530FFF79EFFD8E70A48DA
:109B740000231A4685210088FFF794FFD0E70648A2
:109B840000231A4619460088FFF790FFC8E700BF74
:109B9400AC2A002058CD0200162B00207C35002072
:109BA40062CD02000C4B4A881B889A4212D10A8863
:109BB40040F677239A420DD18B88084A0849033B23
:109BC4009BB21380074A108800041A4640F0030031
:109BD400FCF7DEBE704700BF162B0020142B0020BC
:109BE4006FCD0200AC2A002008B503784BB9054BB1
:109BF4003B211888FFF750FF18B1BDE80840FDF776
:109C040025B908BD162B0020072808B513D00A284B
:109C14000DD0042819D10D4B13211888FFF73CFFF0
:109C240030F0080311D0BDE80840FDF70FB9BDE8D6
:109C34000840FFF741BF054B1A884FF6FF739A425D
:109C440003D1034800F0CDFEEAE708BD162B00203F
:109C5400AC34002008B548B103280BD10220FFF72B
:109C6400F9FD38B1BDE80840FDF7F0B8BDE808409B
:109C7400FFF722BF08BD00000378012BF7B52FD0F2
:109C840003D3022B2CD003B0F0BD174C174D207812
:109C94002844FDF7C7FC23780133DBB21D4423704D
:109CA40015F8012C0A2A03D0114A12889A42EAD8DC
:109CB400104D0E4E104F237802AA314622F8023D71
:109CC40038462B8801F004FC082806D01128F2D06D
:109CD400052802D008B1FDF7B9F800232370D2E7B4
:109CE4004068FDF7B3F8CEE7A8340020B433002071
:109CF400142B0020162B0020182B00202DE9F041F6
:109D0400047805462CBB144FDFF85080AA8A94428D
:109D14000AD32B69134413F8013C0D2B19D10A20E3
:109D2400FDF796FC1128F9E72B69185DFDF790FC07
:109D3400064660B11128F7D03888000440F00100CD
:109D440032464146FCF71AFE3046FDF77FF80134EF
:109D5400DCE7BDE8F08100BFAC2A0020D2CD0200D0
:109D6400FDF774B808B50849084801F09BF808B134
:109D7400FDF76CF8F721054801F0A8F818B1BDE823
:109D84000840FDF763B808BDA99B020064350020B4
:109D940000B5794D0FCDB1B005AC0FC495E8030003
:109DA400764B774A01934FF4807384E8030002935F
:109DB40003920493734A072301A905A8FDF7DAFB6C
:109DC40008B1FDF743F84FF400410020FCF70AFC0A
:109DD40008B1FDF73BF8FCF72FFBFDF7B5FA08B126
:109DE400FDF734F868490320FFF740FD08B1FDF79B
:109DF4002DF805A90020FFF72FFE08B1FDF726F87E
:109E0400FEF70AF908B1FDF721F801F0F5FB08B1F6
:109E1400FDF71CF8002305A90120059301F0C0FCFF
:109E240008B1FDF713F805A801F082FD08B1FDF7AC
:109E34000DF89DF804305548012262F3030362F3E0
:109E440007138DF8043001F09DFF504982B201A838
:109E5400FFF726FE08B1FCF7F9FF0822002105A848
